:020000040000FA
:020000000428D2
:08000800FF30A100EA20EF2007
:1000100000300321A11502212210FE20A210FD2094
:100020002211FC20A301A401A501A601A701A8019A
:10003000A901AA01AB01AC01AD01AE01AF01AB0159
:100040002B08B000F3203108AD000130AE002E08BF
:10005000B000F3203108AF002F08AB00C9202408FE
:100060002702031D7D2825082802031D7D2823085B
:100070002602031D7D282B08B000F3203108AC00B8
:10008000AB0A2C08B000E2203108A9003208A60013
:10009000A908031959282B08B000F3203108AC0037
:1000A000AB0A2C08B000E2203108A7003208A800F3
:1000B00075282F08AB002B08B000F3203108AC00E6
:1000C000AB0A2C08B000E2203108A9003208A600D3
:1000D0002B08B000F3203108AC00AB0A2C08B000AC
:1000E000E2203108A7003208A8002908B100033037
:1000F000B2001621B0003008A90023082602031818
:10010000852801302302A3008A2826082302031829
:100110008A28A30A240827020318922801302402FF
:10012000A40097282708240203189728A40A250862
:10013000280203189F2801302502A500A4282808BA
:1001400025020318A428A50A2908B000B008031D39
:10015000AA28C728AA011030B100221023082A02B9
:100160000318B3282214FE20A21024082A02031820
:10017000BA28A214FD20221125082A020318C1283A
:100180002215FC20AA0AB10BAD28B003A6282E2800
:10019000C8288519E1288519CE28CB2801300821E7
:1001A0008519D328D028AE0A2E082D020318DA2884
:1001B0000130AE002E08B000F3203108AF002F0848
:1001C000AB000800B200300E0F39B10030080F3913
:1001D000B20008008316FF239000831208008316E4
:1001E0009F0183120800B100300883169B001C1485
:1001F0001A088312B1000800FF28FF28FF282208F0
:10020000850008000529A1000529210865000800CE
:10021000B0009E30B1001030B200B10B1029B20B0B
:100220000D2912291329B00B09290800B200320840
:10023000003C031C1C2922290310B10D013032029D
:08024000B20017293108080083
:10420000030004000B0018004F0000004000F00005
:1042100040000F000000600000006F000000600020
:1042200000006000F0006000000060000F0000006F
:0A423000200000002F00FF00000036
:02400E0084111B
:00000001FF
